:020000040000FA
:100000008D01860185018316F0308600023085005F
:100010003730810083128B010516252203308600BC
:100020003C2218223C2218223C2218220230860050
:100030003C2228302D2206302D220C302D22432246
:10004000861B3F280F30D8204F2001300C1C023077
:10005000302203010C1C02309000CF20A5204F203D
:100060000C1E9D208C1EA1208D1C2F28340888007A
:100070001008E620890A35088800E7201F28432257
:100080004F2041220C1D68288C188C1D49284322C2
:100090003B2943308C1C4C3032226420402883168C
:1000A000FF3086008312182206088C008316F03079
:1000B000860083128D100C080D060139031D8D1466
:1000C0000D100C180D140800C0302D222030322ADB
:1000D0000D1343221D30D8204C2282302D220C18C3
:1000E0009320A0220C1C77283E08302278284A2230
:1000F0003D300F223D300F2246223C300F223C3053
:100100000F22C0302D2214221422162216224A2237
:100110000430D82082302D224F200C1D6C28432221
:100120008D1F3F28672906308E000310AE0DAD0DE0
:10013000AC0DAB0D8E0B95280800B50A0319B40A57
:10014000A528B5080319B403B5033230BD20A02299
:100150008B302C2214220C1C46221422162216222A
:100160004A2225220800233092002B309300C02819
:100170002B3093003230BF28273093002B30920071
:1001800004308E00130884000008940012088400D4
:1001900014088000920A930A8E0BC228080083126A
:1001A0008900F720E120B400890AE120B5000800A9
:1001B00089000908E120FF39031908003222890A61
:1001C000D9288316081483120808080089008316AA
:1001D000081555308900AA3089008814081188183C
:1001E000EF28831208000F3084004130FC283230A1
:1001F000FA282B30840004308E008001840A8E0B94
:10020000FD2808008D1A67290D174C224629363023
:10021000B420BC203630B9201B211F30B9209823D0
:1002200096212330B9203630BD20982382302D22EC
:100230008C14A2296729FF22B820B230AB006630A7
:10024000AC006030AD00B130AE003C2302302F2155
:10025000F7208A30B2007A30B3003C230800CF2068
:100260003421C822FF2208001B30B4203230BD20C8
:100270001B30B920080043220830D8204C229001BE
:1002800009302622F3204C224330B4202730B420FA
:10029000051425226420093026224C223630B42051
:1002A000B8200510BC209823B8203630BD203C2350
:1002B00003012F210D1B0729B320B820BC201B21CF
:1002C0001F30B42043222030D82064208D174F20C7
:1002D0000C1D68288C188C1D7329901B3B29900AD3
:1002E000FF301E2267294122773090008D180229A5
:1002F0004C228C1882298D1E80290D1B43220D1340
:100300000D1B0A290D1B43220D13B8204330BD20BD
:100310003C23F7208130B20098232B08031D91293C
:10032000F9208C189C291F30B920FF221A30D820C0
:100330008D1E9B29F920A1292330B920FF221730D7
:10034000D820642091012B08803C0318AF29F720A6
:100350008430B2002030B3003C23910AA3298E30B0
:10036000B2001C30B3004030B400B501FF22ED22D2
:10037000A0221108AB0075309800703097002B0850
:10038000031DCA2948224622142214228C18FC2953
:100390001622FD29AB0BD429142246221422162240
:1003A0008C18FC291622FD29AB0BDC2914221422FF
:1003B000462216221622FD29AB0BE4291422142210
:1003C000162246221622FD296D3098006E309700C5
:1003D000AB0BF02914224622142216221622FD29E4
:1003E000E430AB0BF429D629AB0BF729DE292030FA
:1003F0009800AB0BD629CC294A228C18072A18085A
:100400003222483032224A220D1B08006729170881
:1004100032220D1B6729463032224A226729840086
:10042000800E0008302208003B300F2A3A300F2A95
:1004300007301E2A3F309A0001301F2A9A01990086
:100440009A0B202A990B202A080002309B00FF30CB
:100450001E229B0B272A0800C03095000511342A64
:100460000F39303895000515150E0F3986008515A2
:10047000851115080F3986008515851186011A2208
:1004800008000230442A01302D22182A2E30322A48
:100490003030322A2030322AC001BF018B01810165
:1004A00029300C1DCE308F00831612308500831248
:1004B00016308E008B221A228E0B5A2A00008F0BC8
:1004C000582A3C300C1DB4308E008B22672A8B22B8
:1004D0008E0B652A83160230850083128B22010859
:1004E000C100C20183160116000001128312C2036B
:1004F000010841060319722A3F30BD208D12F030E9
:1005000042054104400403198D160C1D0800C82241
:10051000B820FF2208000B1D9A2AFF300311400269
:10052000031D962ABF0AC0010B119F2AC00A0B1196
:1005300000009F2A00009C2A9D2A9E2A9F2A0800CC
:1005400020309A00BA01BB01BC01BD01BE01AE0D55
:10055000AD0DAC0DAB0DBA0DBB0DBC0DBD0DBE0D83
:100560009A0BB32A080005308F003A308400B92A6C
:10057000840ABD228F0BB82AA72A033000079900EE
:1005800099198000303000079900991B80000800FD
:100590009830AB00960199012C08031DE02A2D0824
:1005A000AC002E08AD00AE0199152C08031DE02A01
:1005B0002D08AC00AD01991119162C080319FD2A5C
:1005C0001908AB020310AC1BEA2AAE0DAD0DAC0D41
:1005D000AB03E32A961FAC130034AC178030AB0298
:1005E000AB1F0319FD2A2B08183CAB000310AC0C01
:1005F000AD0CAE0CAB0BF62A0034F92000342B08FE
:10060000031D32080319FD2A2C0833069600320810
:10061000AB078030031C0E2BAB070F2BAB07AC17BF
:10062000B3170310AF01B001B101183099002E1CAF
:10063000232B3508B10734080318340FB0073308EB
:100640000318330FAF07AF0CB00CB10CAC0CAD0CF2
:10065000AE0C0310990B172BAF1B332BAC0DB10D48
:10066000B00DAF0DAB03961FAF132F08AC003008D1
:10067000AD003108AE0000342C0833069600AC17EC
:10068000B31799012C08AF002D08B0002E08B10057
:100690003508B1023408031C340FB0023308031CC0
:1006A000330FAF02AF01B001B101031C5E2B031089
:1006B000AC0CAD0CAE0CAF0C013099003208AB02A3
:1006C000031C662B80301907AB07692B8030190794
:1006D000AB0718309A00B10DB00DAF0DAE0DAD0DDA
:1006E000AC0D990D3508AE023408031C340FAD0271
:1006F0003308031C330FAC02330D9904191C822BF1
:1007000031148D2B3508AE0734080318340FAD07AC
:1007100033080318330AAC0731109A0B6B2B961F62
:10072000AF132F08AC003008AD003108AE00003424
:100730003208031D9E2B3308031900348030B306A2
:100740002C08330699002B083202031CA82B3421F5
:100750002C089600AC17B3173308AF003408B0006C
:100760003508B10032082B02B2000319D42B08302F
:100770003202031CCB2BB200B10D3008B1002F08A0
:10078000B000AF0108303202031CCB2BB200B10D18
:100790003008B100B00132080319D42B0310AF0C9C
:1007A000B00CB10CB20BCE2B991FDE2BAF09B009E8
:1007B000B109B10A0319B00A0319AF0A3108AE072B
:1007C00030080318300FAD072F0803182F0FAC07A0
:1007D000991BF12B031CEA2AAC0CAD0CAE0CAB0A36
:1007E000EA2A0318CB2AAC09AD09AE09AE0A0319EF
:0C07F000AD0A0319AC0A80309606CB2A33
:02400E00F13F80
:104200000300E8000300E8004D0048007A000000C9
:1042100020002000570041004900540000004300E6
:104220006F006E007300740020005800000043000F
:104230003D0000004C003D00000046003D00000035
:064240004F004B000000DE
:00000001FF
